:020000040000FA
:020000000C28CA
:08000800A0000308A10021087B
:100010008300A00E200E0900FF23831690008B01A1
:100020006400DB3081006400203084003F308001B8
:10003000840AFF3E031D17280B30850053309F00B4
:10004000831283309F000030DD002E30DE0001304F
:10005000DF0041212E082E072E07013EDD0028304B
:10006000DE000330DF004121AE0A28302E020319E2
:10007000AE012E30DD000030DE000130DF004D210A
:1000800028080C21A50029080C21A6002A080C210B
:10009000A7005030DC006400AC0A40302C02031D85
:1000A0005F28AC01DC0B5F281E0883161E08831234
:1000B000A801A501A901A601AA01A70163280A3088
:1000C0000721D9204B286400AC0A40302C02031DC4
:1000D000D528AC012A080C21A7002B08031D76287F
:1000E0002A08031D7E280130AB007C28FF302A023D
:1000F000031D7C28AB017E28AA0A7F28AA03831649
:100100002A1C93281E0803198A2829070318FF3080
:10011000A9008F2829080319A3282221A90029084A
:100120000C21A600A3281E0803199B2828070318E2
:10013000FF30A800A02828080319A3282221A8001E
:1001400028080C21A5008312A508031DCE28A608A7
:10015000031DCE28AD0A32302D02031DCF281F10FB
:1001600034308500640063001F1401300721103013
:10017000AD0083309F004B30072183169E08831209
:10018000031DCE2883309F004B30072183169E0825
:100190008312031DCE28AD0BB928AF28AD012A1C50
:1001A000D3288730D42883309F000A300721D920F4
:1001B00063282208031DE728051DE22805112508EC
:1001C000A200E82805152508FF3AA200E828A203A6
:1001D0002308031DF628051EF12805122608A30092
:1001E000F72805162608FF3AA300F728A3032408DA
:1001F000031D0529851E002985122708A40006294C
:1002000085162708FF3AA4000629A4030800DB008E
:100210006400DB0B08290800DB00803C031C152967
:10022000DB0CDB0C3F305B0521295B08C03C031C69
:100230001C2960305B022129C030DB02DB0D6030FD
:100240005B070800DB00803C031C282901302F29B4
:100250005B08C03C031C2E2902302F2904305B02AE
:1002600008009B001C141A08080055309D00AA3095
:100270009D009C140730DC00FA300721DC0B3C2980
:10028000080083165E0884005D0831218000DD0AC5
:10029000840ADF0B44298312080083161C155D08AD
:1002A00084005E089B0000089A0035211A081C147F
:1002B0001A06031D6329840ADE0ADF0B51291C116B
:0A02C00083120130642903010800D5
:02400E00AC3FC5
:104200000000FA0041002F00260079002100E9009B
:104210007B00AF00CA004D002E009300CC00D600FA
:10422000500087005000A7005F00DE00A900A90031
:10423000EF00F800AF002600AE0021007C008F00E8
:10424000D0005000A800F6006400A2005E007700D5
:10425000E0008500E700C600F7009300DC0088005E
:104260004E00750045001500E900C700CE0047006C
:104270006600AD002B003800A300C700F5007E00EB
:10428000D400C6001D00A60070003200F500F0004A
:1042900079000B00E000C400D300270095009200D5
:1042A000B7004600C300040022005900F400FA00E1
:1042B00086002B0085004F002F004500D0009B009A
:1042C0000A0075006C0007001600E6002E0078005A
:1042D000320012000B0025005C003000AC009A0098
:1042E000C800FD006B00650027008800FB00570038
:0242F0001600B6
:00000001FF
